:100000000C948F000C94AA000C94AA000C94AA00E3
:100010000C94B1070C94BD060C9484070C942A0729
:100020000C9457070C9490060C94FD060C943D0616
:100030000C94AA000C94AA000C94AA000C94AA0098
:100040000C94AA000C94AA000C94AA000C94AA0088
:100050000C94AA00001F000000001F00001F1010D9
:1000600010101F00001F181818181F00001F1C1C5C
:100070001C1C1F00001F1E1E1E1E1F00001F1F1F16
:100080001F1F1F0003070F1F0F070300001F1F1F65
:100090001F1F1F001B1B1B1B1B1B1B00181C1E1FD5
:1000A0001E1C18000004040E0E1F1F00001F1F0E50
:1000B0000E0404000000000000000000000E1915EE
:1000C000130E0000000E1515150E0000000E13157E
:1000D000190E0000000E111F110E000030313233D6
:1000E0003435363738394142434445460000000133
:1000F000000800400000010004000001000800208A
:1001000000400080000001000448656C6C6F20779F
:100110006F726C642E2020202020202020001124CB
:100120001FBECFE5D8E0DEBFCDBF10E0A0E6B0E057
:10013000EAE7F1E102C005900D92A036B107D9F7C8
:1001400010E0A0E6B0E001C01D92AE37B107E1F7C4
:100150000C942E080C940000C298C198C398BA9AC7
:10016000B99ABB9A87B38F7087BB88B3806F88BBFF
:100170000895C29887B38F7087BB88B3806F88BBA0
:10018000C19AC39A0000000000000000B79B26C07F
:10019000C398000000000000000000000000000004
:1001A0000000C39A000000000000000000000000F2
:1001B00000000000C39800000000000000000000E4
:1001C000000000000000C39A0000000000000000D2
:1001D0000000000000000000B799DACFC39808952E
:1001E0001F93182F0E94B900C298C198C39A87B371
:1001F000806F87BB88B38F70912F907F892B88BBCE
:1002000000000000000000000000000000000000EE
:10021000C398000000000000000000000000000083
:100220000000C39A28B32F70812F992734E0880FDC
:10023000991F3A95E1F7282B28BB00000000000029
:1002400000000000000000000000C39887B38F701A
:1002500087BB88B3806F88BB1F9108950E94B90047
:1002600087B38F7087BB88B3806F88BBC298C19AF1
:10027000C39A000000000000000000000000000021
:10028000000096B3907FC3980000000000000000BB
:100290000000000000000000C39A00000000000001
:1002A0000000000000000000000086B382958F70FF
:1002B000982BC398892F992708951F93182F0E9470
:1002C000B900C29AC198C39A87B3806F87BB88B3BD
:1002D0008F70912F907F892B88BB00000000000059
:1002E00000000000000000000000C39800000000B3
:1002F000000000000000000000000000C39A28B3C6
:100300002F70812F992744E0880F991F4A95E1F7B4
:10031000282B28BB000000000000000000000000A7
:1003200000000000C39887B38F7087BB88B3806FCD
:1003300088BB1F9108950E94B90087B38F7087BB57
:1003400088B3806F88BBC29AC19AC39A000000002C
:1003500000000000000000000000000096B3907F45
:10036000C398000000000000000000000000000032
:100370000000C39A00000000000000000000000020
:100380000000000086B382958F70982BC398892F48
:1003900099270895AF92BF92CF92DF92FF920F9369
:1003A0001F93CF93DF93CDB7DEB721970FB6F894A5
:1003B000DEBF0FBECDBF6C01062F142F0E942E0191
:1003C0008F778983110F110F110F000F000F000F8E
:1003D000FF24AA24BB24812F8F0D80640E94F0008B
:1003E000F601E00FF11DEA0DFB1D84910E945D01F5
:1003F000F3940894A11CB11C87E08F1560F78981E4
:1004000080680E94F00021960FB6F894DEBF0FBE00
:10041000CDBFDF91CF911F910F91FF90DF90CF90D3
:10042000BF90AF9008950E94AC0088E20E94F00057
:1004300081E00E94F00080E69AEE0E94080586E0C6
:100440000E94F0008CE00E94F00082E00E94F00028
:1004500080E80E94F00040E0642F84E590E00E9474
:10046000CA0141E0642F84E590E00E94CA0142E0A5
:10047000642F84E590E00E94CA0143E0642F84E584
:1004800090E00E94CA0144E0642F84E590E00E945D
:10049000CA0145E0642F84E590E00E94CA0146E06D
:1004A000642F84E590E00E94CA0147E0642F84E550
:1004B00090E00E94CA01089582E00E94F000089531
:1004C00081E00E94F0000895282F862F992781301F
:1004D000910549F0823091057CF08230910531F030
:1004E000039739F009C0822F805C07C0822F8C5E91
:1004F00004C0822F8C5A01C0822F80680E94F000B5
:1005000008950F931F93CF93009759F0662349F0F6
:100510008C01C62FF80181918F010E945D01C150AD
:10052000C9F7CF911F910F910895DF92EF92FF923B
:100530000F931F93CF93DF93242F3327829FF001D4
:10054000839FF00D929FF00D1124CF01880F991F0A
:10055000880F991F8E0F9F1F8E0F9F1F0E946C0880
:100560007B0100271127442349F1C0E0D0E0D42EBD
:100570002596CE01AA27BB272597E816F9060A0774
:100580001B07A8F4CE01AA27BB27E816F9060A071D
:100590001B0710F480E00CC0C801B70126E030E072
:1005A00040E050E00E948008DC01CB0101C085E002
:1005B0000E945D01DA942696DD20D1F6DF91CF917D
:1005C0001F910F91FF90EF90DF900895909361003D
:1005D000809360000895E0916000F09161000995BA
:1005E0000895CF93DF93EC01892B61F088818823F4
:1005F00049F0E0916000F09161008991099588814E
:100600008823B9F7DF91CF910895EF92FF920F936E
:100610001F93CF93DF93EC017A0120E030E0892B28
:1006200001F1C9012F5F3F4F8617970718F4899191
:100630008823B9F720E030E02E153F0590F488813B
:1006400089010F5F1F4FE0916000F09161008823E6
:1006500011F0219601C080E2099598010E151F0541
:1006600070F3DF91CF911F910F91FF90EF9008955C
:10067000CF93DF93EC01009779F0FC0121968491F0
:10068000882351F0E0916000F09161000995FE012E
:10069000219684918823B1F7DF91CF910895E0915D
:1006A0006000F09161008DE00995E0916000F091AB
:1006B00061008AE009950895E82FFF27EF70F07038
:1006C000E452FF4F8491E0916000F0916100099540
:1006D00008951F93182F82958F700E945C03812FBD
:1006E0000E945C031F9108950F931F938C01812F2B
:1006F00099270E946903802F0E9469031F910F911F
:100700000895EF92FF920F931F937B018C01C80114
:10071000AA27BB270E947403C7010E9474031F917C
:100720000F91FF90EF9008952F923F924F925F921A
:100730006F927F928F929F92AF92BF92CF92DF92F1
:10074000EF92FF920F931F93CF93DF93CDB7DEB756
:10075000A2970FB6F894DEBF0FBECDBF69A3C42E1B
:100760002AA327013801442351F017FF08C0EE24C3
:10077000FF248701E418F5080609170902C0830160
:10078000720199A1692F772767FD709561507040BC
:10079000CC2011F061507040D62E18A22FE1222EED
:1007A000312C2C0E3D1E882E992487FC9094A92C68
:1007B000B92CC801B701A50194010E948008DC0191
:1007C000CB01FC01E452FF4F84918F8FC801B70128
:1007D000A50194010E94800879018A01DA94AFEFA3
:1007E000DA1639F1DA94C1010197E114F104010537
:1007F0001105C1F01C01C801B701A50194010E94B7
:100800008008DC01CB01FC01E452FF4F8491F1012F
:100810008083C801B701A50194010E948008790175
:100820008A0104C01C01EAA1DC01EC93FFEFDF1692
:10083000C9F6CC20B9F077FE05C08DE2D1018E93C8
:100840001D0110C0C10101971414150416041704EA
:100850002CF41C018BE2F101808304C01C0180E2B6
:10086000D1018C93D9A0DA94BFEFDB1661F0E0914F
:100870006000F0916100D1018D911D010995DA941C
:10088000BFEFDB16A1F7A2960FB6F894DEBF0FBE3E
:10089000CDBFDF91CF911F910F91FF90EF90DF902F
:1008A000CF90BF90AF909F908F907F906F905F9010
:1008B0004F903F902F9008957F928F929F92AF928A
:1008C000BF92CF92DF92EF92FF920F931F93CF933D
:1008D000DF93CDB7DEB77888C988DA8863E1A62EC2
:1008E000B12CAC0EBD1E08C0882309F481C0E09174
:1008F0006000F0916100099596012F5F3F4F7720CE
:1009000021F0F6016901849103C0F601808169013B
:10091000853251F72F5F3F4F772021F0F6016901B3
:10092000849103C0F60180816901282F332727FDB8
:1009300030952436310591F02536310524F42336DF
:10094000310529F0D4CF2837310581F0D0CFF5011A
:1009500022E030E0A20EB31E8081C9CF5AE0852E7E
:10096000912C40E1E42E47E2F42E04C030E1E32E66
:10097000F12C4701F50122E030E0A20EB31E008108
:1009800011818436D9F417FF09C0109501951F4FC6
:10099000E0916000F09161008DE2099532E0E3168C
:1009A000F10460F00E151F0548F4C7016AE070E01D
:1009B0000E946C087B0162307105A0F7C801B70185
:1009C0000E946C08FB01E452FF4F8491E0916000AB
:1009D000F09161000995C801B7010E946C088C0173
:1009E000C701B4010E946C087B01672B39F784CFE3
:1009F00080E090E0DF91CF911F910F91FF90EF90F9
:100A0000DF90CF90BF90AF909F908F907F90089590
:100A1000089593B7987F982B93BF08959EB5987FBC
:100A2000982B9EBD089595B5987F982B95BD0895F8
:100A3000E3B7FF27E770F070EE0FFF1FE351FF4FA2
:100A4000859194910895EEB5FF27E770F070EE0F51
:100A5000FF1FE351FF4F859194910895E5B5FF275E
:100A6000E770F070EE0FFF1FE750FF4F85919491F4
:100A70000895883040F4E82FFF27EE0FFF1FEE594E
:100A8000FF4F718360830895883040F4E82FFF277B
:100A9000EE0FFF1FEE59FF4F118210820895DF9273
:100AA000EF92FF920F931F937C01D2B610927600C3
:100AB0001092770010927800109279000E94180529
:100AC0009C014427552760E074E284EF90E00E9487
:100AD000A208293B8DE8380786E0480780E05807E0
:100AE00098F481E1E81687E2F80670F4B7018827E8
:100AF00099270E944D0828EE33E040E050E00E9424
:100B0000800879018A0123C000271127CA01B90191
:100B100028EE33E040E050E00E948008C801B701B1
:100B20000E944D087B018C0112C08091760090914B
:100B30007700A0917800B091790085B78F7885BF54
:100B400085B7806885BF889585B78F7785BF809189
:100B5000760090917700A0917800B091790022B74B
:100B6000BA2FA92F982F8827332744275527822B60
:100B7000932BA42BB52BA80197012D0D311D411DE1
:100B8000511D82179307A407B50778F21F910F91A3
:100B9000FF90EF90DF900895109272001092730012
:100BA0001092740010927500089560917200709117
:100BB00073008091740090917500089510927A00EE
:100BC00010927B0010927C0010927D00089560913D
:100BD0007A0070917B0080917C0090917D00089557
:100BE000893031F48FB582608FBD8FB58E7F0AC09A
:100BF0008A3019F48FB5826002C08FB58D7F8FBDAA
:100C00008FB581608FBD1BBC1ABC19BC18BC089580
:100C10002FB52E7F2FBD2FB522602FBD2EB528609A
:100C20002EBD2EB520612EBD97BD86BD1BBC1ABC46
:100C300019BC18BC08958FB580688FBD8FB58F7BA8
:100C40008FBD08958FB580628FBD8FB58F7E8FBDAC
:100C500008958FB58F778FBD8FB58F7B8FBD08952A
:100C60008FB58F7D8FBD8FB58F7E8FBD08959BBD56
:100C70008ABD089599BD88BD08951F920F920FB641
:100C80000F9211242F933F934F935F936F937F9312
:100C90008F939F93AF93BF93EF93FF9380917200D5
:100CA00090917300A0917400B09175000196A11D00
:100CB000B11D8093720090937300A0937400B09361
:100CC00075008091760090917700A0917800B091A6
:100CD00079000196A11DB11D809376009093770055
:100CE000A0937800B09379008091620090916300A6
:100CF000892B29F0E0916200F09163000995FF9142
:100D0000EF91BF91AF919F918F917F916F915F9183
:100D10004F913F912F910F900FBE0F901F901895FC
:100D20001F920F920FB60F9211242F933F934F9360
:100D30005F936F937F938F939F93AF93BF93EF9343
:100D4000FF938091640090916500892B29F0E091D8
:100D50006400F09165000995FF91EF91BF91AF910B
:100D60009F918F917F916F915F914F913F912F91C3
:100D70000F900FBE0F901F9018951F920F920FB6F5
:100D80000F9211242F933F934F935F936F937F9311
:100D90008F939F93AF93BF93EF93FF9380917A00CC
:100DA00090917B00A0917C00B0917D000196A11DE7
:100DB000B11D80937A0090937B00A0937C00B09348
:100DC0007D0080916C0090916D00892B29F0E0915D
:100DD0006C00F0916D000995FF91EF91BF91AF917B
:100DE0009F918F917F916F915F914F913F912F9143
:100DF0000F900FBE0F901F9018951F920F920FB675
:100E00000F9211242F933F934F935F936F937F9390
:100E10008F939F93AF93BF93EF93FF938091700055
:100E200090917100892B29F0E0917000F091710090
:100E30000995FF91EF91BF91AF919F918F917F9114
:100E40006F915F914F913F912F910F900FBE0F9037
:100E50001F9018951F920F920FB60F9211242F9387
:100E60003F934F935F936F937F938F939F93AF9332
:100E7000BF93EF93FF938091660090916700892B59
:100E800029F0E0916600F09167000995FF91EF91DC
:100E9000BF91AF919F918F917F916F915F914F9192
:100EA0003F912F910F900FBE0F901F9018951F929A
:100EB0000F920FB60F9211242F933F934F935F938E
:100EC0006F937F938F939F93AF93BF93EF93FF9312
:100ED0008091680090916900892B29F0E091680069
:100EE000F09169000995FF91EF91BF91AF919F91AA
:100EF0008F917F916F915F914F913F912F910F90C3
:100F00000FBE0F901F9018951F920F920FB60F9261
:100F100011242F933F934F935F936F937F938F93FE
:100F20009F93AF93BF93EF93FF9380916A0090914B
:100F30006B00892B29F0E0916A00F0916B00099514
:100F4000FF91EF91BF91AF919F918F917F916F91A1
:100F50005F914F913F912F910F900FBE0F901F9077
:100F600018951F920F920FB60F9211242F933F9353
:100F70004F935F936F937F938F939F93AF93BF93A1
:100F8000EF93FF9380916E0090916F00892B29F071
:100F9000E0916E00F0916F000995FF91EF91BF9184
:100FA000AF919F918F917F916F915F914F913F9101
:100FB0002F910F900FBE0F901F90189583B7887FC9
:100FC000826083BF12BE89B7816089BF10927200B0
:100FD00010927300109274001092750008958EB5EF
:100FE000887F83608EBD1DBC1CBC89B7846089BFAF
:100FF000089585B5887F846085BD14BC89B78064F9
:1010000089BF10927A0010927B0010927C0010929F
:101010007D000895E2E6F0E011821082329680E0D1
:10102000E237F807C9F70E94DE070E94EF070E9427
:10103000F907789408958FB58D7F8FBD8FB58E7F1A
:101040008FBD8FB58F778FBD8FB58F7B8FBD8FB5E0
:101050008F7D8FBD8FB58F7E8FBD0895CFE5D8E092
:10106000DEBFCDBF0E9413028DE591E00E94E60233
:101070000E9460021ABA14BA11BA60E0862F0E9468
:10108000640289E091E09F938F9381E08F930E94A7
:101090005C040F900F900F90FFCF629FD001739F61
:1010A000F001829FE00DF11D649FE00DF11D929F04
:1010B000F00D839FF00D749FF00D659FF00D992743
:1010C000729FB00DE11DF91F639FB00DE11DF91F67
:1010D000BD01CF0111240895AA1BBB1B51E107C01C
:1010E000AA1FBB1FA617B70710F0A61BB70B881FB8
:1010F000991F5A95A9F780959095BC01CD01089547
:10110000A1E21A2EAA1BBB1BFD010DC0AA1FBB1F0B
:10111000EE1FFF1FA217B307E407F50720F0A21B7D
:10112000B30BE40BF50B661F771F881F991F1A94EA
:1011300069F760957095809590959B01AC01BD0114
:10114000CF01089597FB092E05260ED057FD04D038
:10115000D7DF0AD0001C38F4509540953095219582
:101160003F4F4F4F5F4F0895F6F7909580957095DC
:0A11700061957F4F8F4F9F4F089548
:00000001FF
